:100000000C942A000C9445000C9445000C94450077
:100010000C9445000C9445000C9445000C9445004C
:100020000C9445000C9445000C9445000C9447003A
:100030000C9445000C9445000C9445000C9445002C
:100040000C9436010C9445000C9445000C9445002A
:100050000C94450011241FBECFE5D8E0DEBFCDBF14
:1000600010E0A0E6B0E0EAEBF2E002C005900D92ED
:10007000A036B107D9F710E0A0E6B0E001C01D92AC
:10008000A937B107E1F70C949D000C9400001F9272
:100090000F920FB60F9211248F939F93809174004B
:1000A000982F9F5F909374009923A1F4809176001C
:1000B0008093600080916100809375008091620060
:1000C000809363008091770080937800C09AC19AF2
:1000D000C29AC39A80916000981709F4C0988091E1
:1000E0007500981709F4C19880916300981709F476
:1000F000C29880917800981709F4C3989F918F91C6
:100100000F900FBE0F901F90189581E083BF89B7A5
:10011000816089BF08958CEC86B980E090E024E688
:1001200030E0FC01EE0FFF1FE20FF31F118210827F
:10013000019688309105A9F70895CFE5D8E0DEBF94
:10014000CDBF1ABA8FEF87BB14BA11BA10927600DE
:100150001092610010926200109277000E948B0052
:100160000E94850078942091640030916500809110
:10017000660090916700281B390BC90122F488277B
:100180009927821B930B8F3F910519F014F08FEF85
:1001900090E0809376001216130614F4C49A01C0FE
:1001A000C498209168003091690080916A00909114
:1001B0006B00281B390BC90122F488279927821B61
:1001C000930B8F3F910519F014F08FEF90E080931F
:1001D00061001216130614F4C59A01C0C598209147
:1001E0006C0030916D0080916E0090916F00281B23
:1001F000390BC90122F488279927821B930B8F3F63
:10020000910519F014F08FEF90E0809362001216C0
:10021000130614F4C69A01C0C6982091700030915C
:1002200071008091720090917300281B390BC901F5
:1002300022F488279927821B930B8F3F910519F091
:1002400014F08FEF90E0809377001216130614F4E9
:10025000C79A89CFC79887CFFC01E770F070EE0F7F
:10026000FF1FEC59FF4F8081918108951F920F92DB
:100270000FB60F9211242F933F938F939F93EF9379
:10028000FF9387B199278770907024B135B1FC0135
:10029000EE0FFF1FEC59FF4F3183208301968770CB
:1002A00087B9369AFF91EF919F918F913F912F914E
:0A02B0000F900FBE0F901F901895DD
:00000001FF
